:020000020000FC
:1000000091C090C08FC08EC08DC08CC08BC08AC084
:1000100089C088C087C086C085C084C083C082C0B4
:1000200081C080C07FC0E3D071E080E1662403E03E
:10003000802E06E0502E77241DD0002D0F3F51F466
:10004000F2E0E0E0C8951FD0002021F0EF5FFF4F05
:100050007394F8CF92D081507040E0F771E080E166
:1000600027D05A94B9F706E0502E17D0882091F780
:10007000969AFECF0FB7F894E199FECF7EBAE09A38
:100080000DB20FBF08950FB7F894E199FECF7EBA75
:100090000DBAE29AE19A0FBF0895762CEBDF6394D4
:1000A000002021F4662400E2002E8A9413D00895E3
:1000B00008E0302EF0E0E0E602810695028301813F
:1000C00007950183008107950083EC5FFF4F3A9409
:1000D00099F7089500E2001AFF27E02DEE0FFF1FA9
:1000E0000E2F1F2FEE0FFF1FE00FF11F02E212E095
:1000F000E00FF11FEC5FFF4F05E0302E07E0402ED0
:100100001491D0E0C0E6110F0A81001F0A83C39545
:10011000C395C395C3954A94B1F7E150F0403A9422
:1001200069F708950FED0DBF0FE707BB0CE701BBA3
:100130000FEF08BB03E002BB00E00BBF00E009BF0C
:1001400000E005BF04E003BF00E00FBD00E00EBD0E
:1001500000E001BD00E00AB90EE003B901E009B911
:1001600000E002B900E808B97894969894989398BA
:100170009298929A939A929856CFE22DE770EE0F4A
:10018000EE0FFF27E05AFF4F00E1302E0081118172
:10019000001F111F959808F4959A949A94983A9490
:1001A000B9F700E008BB9298929A02D02394089580
:1001B000EF93FF930F93E22DE770EE0FFF27EE51C1
:1001C000FF4F099401E00EC002E00CC004E00AC039
:1001D00008E008C000E106C000E204C000E402C07C
:1001E00000E800C008BB0F91FF91EF91089500E275
:1001F000302EF0E0E0E6002701933A94E9F7089505
:1002000057656C636F6D6520746F2045415369209D
:100210004C696E652041544578706F20323030361D
:1002200000000000000000000000FA00000000E0F4
:1002300000E0000028FE28FE28002454FE54480058
:10024000C4C8102646006C92AA440A0000A0C00050
:10025000000000384482000000824438000028106A
:100260007C10280010107C101000000A0C00000008
:1002700010101010100000060600000004081020E6
:1002800040007C8A92A27C000042FE02000042866E
:100290008A9262008482A2D28C00182848FE08004C
:1002A000E5A2A2A29C003C5292920C00808E90A0EB
:1002B000C0006C9292926C00609292947800006CF4
:1002C0006C000000006A6C000000102844820000EE
:1002D00028282828280000824428100040808A907E
:1002E00060004C929E827C007E8888887E00FE9210
:1002F00092926C007C8282824400FE8282443800AA
:10030000FE9292928200FE90909080007C82929267
:100310005E00FE101010FE000082FE82000004024B
:1003200082FC8000FE1028448200FE0202020200CD
:10033000FE403040FE00FE201008FE007C828282DB
:100340007C00FE90909060007C828A847A00FE900F
:1003500098946200629292928C008080FE8080006D
:10036000FC020202FC00F8040204F800FC021C0279
:10037000FC00C6281028C600E0100E10E000868B96
:1003800092A2C20000FE8282000000000000000075
:10039000008282FE00002040804020000202020213
:1003A0000200008040200000042A2A2A1E00FE12BB
:1003B00022221C001C22222204001C222212FE00E7
:1003C0001C2A2A2A1800107E90804000304A4A4A8F
:1003D0007C00FE1020201E000022BE02000004024D
:1003E00022BC0000FE08142200000082FE02000071
:1003F0003E2018201E003E1020201E001C2222221B
:100400001C003E2828281000102828183E003E1006
:1004100020201000122A2A2A040020FC22020400B4
:100420003C0202043E003804020438003C020C0284
:100430003C00221408142200300A0A0A3C0022263A
:100440002A32220000106C8200000000FE00000032
:0604500000826C100000A8
:00000001FF
